 redefclass030

 Timestamp is 700a2c9e (reproducible build file hash)

 Preferred load address is 0000000180000000

 Start         Length     Name                   Class
 0001:00000000 000039c0H .text$mn                CODE
 0001:000039c0 00000036H .text$mn$00             CODE
 0001:000039f6 00000092H .text$x                 CODE
 0002:00000000 000001d0H .idata$5                DATA
 0002:000001d0 00000038H .00cfg                  DATA
 0002:00000208 00000008H .CRT$XCA                DATA
 0002:00000210 00000008H .CRT$XCZ                DATA
 0002:00000218 00000008H .CRT$XIA                DATA
 0002:00000220 00000008H .CRT$XIC                DATA
 0002:00000228 00000008H .CRT$XIZ                DATA
 0002:00000230 00000008H .CRT$XLA                DATA
 0002:00000238 00000008H .CRT$XLZ                DATA
 0002:00000240 00000008H .CRT$XPA                DATA
 0002:00000248 00000008H .CRT$XPZ                DATA
 0002:00000250 00000008H .CRT$XTA                DATA
 0002:00000258 00000008H .CRT$XTZ                DATA
 0002:00000260 00000000H .gehcont$y              DATA
 0002:00000260 00000000H .gfids$y                DATA
 0002:00000260 000024a0H .rdata                  DATA
 0002:00002700 00000000H .rdata$CastGuardVftablesA DATA
 0002:00002700 00000000H .rdata$CastGuardVftablesC DATA
 0002:00002700 00000028H .rdata$T                DATA
 0002:00002728 000000f8H .rdata$voltmd           DATA
 0002:00002820 00000320H .rdata$zzzdbg           DATA
 0002:00002b40 00000008H .rtc$IAA                DATA
 0002:00002b48 00000008H .rtc$IZZ                DATA
 0002:00002b50 00000008H .rtc$TAA                DATA
 0002:00002b58 00000008H .rtc$TZZ                DATA
 0002:00002b60 00000004H .tls                    DATA
 0002:00002b64 00000004H .tls$                   DATA
 0002:00002b68 00000008H .tls$ZZZ                DATA
 0002:00002b70 00000390H .xdata                  DATA
 0002:00002f00 00000464H .edata                  DATA
 0002:00003364 0000008cH .idata$2                DATA
 0002:000033f0 00000018H .idata$3                DATA
 0002:00003408 000001d0H .idata$4                DATA
 0002:000035d8 0000048eH .idata$6                DATA
 0003:00000000 00000090H .data                   DATA
 0003:00000090 0001b258H .bss                    DATA
 0004:00000000 000003fcH .pdata                  DATA

  Address         Publics by Value              Rva+Base               Lib:Object

 0000:00000000       __AbsoluteZero             0000000000000000     <absolute>
 0000:00000000       ___safe_se_handler_count   0000000000000000     <absolute>
 0000:00000000       ___safe_se_handler_table   0000000000000000     <absolute>
 0000:00000000       __arm64x_extra_rfe_table   0000000000000000     <absolute>
 0000:00000000       __arm64x_extra_rfe_table_size 0000000000000000     <absolute>
 0000:00000000       __arm64x_native_entrypoint 0000000000000000     <absolute>
 0000:00000000       __arm64x_redirection_metadata 0000000000000000     <absolute>
 0000:00000000       __arm64x_redirection_metadata_count 0000000000000000     <absolute>
 0000:00000000       __dynamic_value_reloc_table 0000000000000000     <absolute>
 0000:00000000       __enclave_config           0000000000000000     <absolute>
 0000:00000000       __guard_check_icall_a64n_fptr 0000000000000000     <absolute>
 0000:00000000       __guard_eh_cont_count      0000000000000000     <absolute>
 0000:00000000       __guard_eh_cont_table      0000000000000000     <absolute>
 0000:00000000       __guard_fids_count         0000000000000000     <absolute>
 0000:00000000       __guard_fids_table         0000000000000000     <absolute>
 0000:00000000       __guard_iat_count          0000000000000000     <absolute>
 0000:00000000       __guard_iat_table          0000000000000000     <absolute>
 0000:00000000       __guard_longjmp_count      0000000000000000     <absolute>
 0000:00000000       __guard_longjmp_table      0000000000000000     <absolute>
 0000:00000000       __hybrid_auxiliary_iat     0000000000000000     <absolute>
 0000:00000000       __hybrid_auxiliary_iat_copy 0000000000000000     <absolute>
 0000:00000000       __hybrid_code_map          0000000000000000     <absolute>
 0000:00000000       __hybrid_code_map_count    0000000000000000     <absolute>
 0000:00000000       __x64_code_ranges_to_entry_points 0000000000000000     <absolute>
 0000:00000000       __x64_code_ranges_to_entry_points_count 0000000000000000     <absolute>
 0000:00000100       __guard_flags              0000000000000100     <absolute>
 0000:00000000       __ImageBase                0000000180000000     <linker-defined>
 0001:00000000       ?NewObject@JNIEnv_@@QEAAPEAV_jobject@@PEAV_jclass@@PEAU_jmethodID@@ZZ 0000000180001000 f i libredefclass030.obj
 0001:00000024       ?SetEventNotificationMode@_jvmtiEnv@@QEAA?AW4jvmtiError@@W4jvmtiEventMode@@W4jvmtiEvent@@PEAV_jobject@@ZZ 0000000180001024 f i libredefclass030.obj
 0001:0000002c       ?TranslateError@@YAPEBDW4jvmtiError@@@Z 000000018000102c f   libredefclass030.obj
 0001:000002e4       ?nsk_jni_check_exception@@YAHPEAUJNIEnv_@@QEBDH@Z 00000001800012e4 f   libredefclass030.obj
 0001:00000428       ?nsk_jni_lverify@@YAHHPEAUJNIEnv_@@HQEBDH1ZZ 0000000180001428 f   libredefclass030.obj
 0001:000004c8       Agent_Initialize           00000001800014c8 f   libredefclass030.obj
 0001:000007bc       Agent_OnAttach             00000001800017bc f   libredefclass030.obj
 0001:000007bc       Agent_OnLoad               00000001800017bc f   libredefclass030.obj
 0001:000007c4       CompiledMethodLoad         00000001800017c4 f   libredefclass030.obj
 0001:00000944       CompiledMethodUnload       0000000180001944 f   libredefclass030.obj
 0001:000009f8       Java_nsk_jvmti_RedefineClasses_redefclass030_isRedefinitionOccurred 00000001800019f8 f   libredefclass030.obj
 0001:00000a28       Java_nsk_jvmti_RedefineClasses_redefclass030_notifyNativeAgent 0000000180001a28 f   libredefclass030.obj
 0001:00000a5c       Java_nsk_jvmti_RedefineClasses_redefclass030_storeClassBytes 0000000180001a5c f   libredefclass030.obj
 0001:00000aa4       Java_nsk_jvmti_unit_FollowReferences_FollowRefObjects_addRefToVerify 0000000180001aa4 f   libredefclass030.obj
 0001:00000c60       Java_nsk_jvmti_unit_FollowReferences_FollowRefObjects_getTag 0000000180001c60 f   libredefclass030.obj
 0001:00000d1c       Java_nsk_jvmti_unit_FollowReferences_FollowRefObjects_resetRefsToVerify 0000000180001d1c f   libredefclass030.obj
 0001:00000d24       Java_nsk_jvmti_unit_FollowReferences_FollowRefObjects_resetTags 0000000180001d24 f   libredefclass030.obj
 0001:00000d68       Java_nsk_jvmti_unit_FollowReferences_FollowRefObjects_setTag 0000000180001d68 f   libredefclass030.obj
 0001:00000fb4       Java_nsk_share_jvmti_ArgumentHandler_getAgentOptionsString 0000000180001fb4 f   libredefclass030.obj
 0001:00001060       Java_nsk_share_jvmti_DebugeeClass_checkStatus 0000000180002060 f   libredefclass030.obj
 0001:000010e8       Java_nsk_share_jvmti_DebugeeClass_resetAgentData 00000001800020e8 f   libredefclass030.obj
 0001:00001148       Java_nsk_share_jvmti_RedefineAgent_agentStatus 0000000180002148 f   libredefclass030.obj
 0001:00001154       Java_nsk_share_jvmti_RedefineAgent_isRedefined 0000000180002154 f   libredefclass030.obj
 0001:00001160       Java_nsk_share_jvmti_RedefineAgent_redefineAttempted 0000000180002160 f   libredefclass030.obj
 0001:0000116c       MA_checkStatus             000000018000216c f   libredefclass030.obj
 0001:00001210       __local_stdio_printf_options 0000000180002210 f i libredefclass030.obj
 0001:00001914       exitOnError                0000000180002914 f   libredefclass030.obj
 0001:000019c8       fprintf                    00000001800029c8 f i libredefclass030.obj
 0001:00001a0c       nsk_complain               0000000180002a0c f   libredefclass030.obj
 0001:00001a38       nsk_jvmti_createJVMTIEnv   0000000180002a38 f   libredefclass030.obj
 0001:00001b68       nsk_jvmti_enableEvents     0000000180002b68 f   libredefclass030.obj
 0001:00001c44       nsk_jvmti_lverify          0000000180002c44 f   libredefclass030.obj
 0001:00001d34       nsk_jvmti_parseOptions     0000000180002d34 f   libredefclass030.obj
 0001:00001f84       nsk_jvmti_resetAgentData   0000000180002f84 f   libredefclass030.obj
 0001:00001ff8       nsk_jvmti_resumeSync       0000000180002ff8 f   libredefclass030.obj
 0001:0000209c       nsk_jvmti_waitForSync      000000018000309c f   libredefclass030.obj
 0001:000021a0       nsk_lcomplain              00000001800031a0 f   libredefclass030.obj
 0001:000021c0       nsk_ldisplay               00000001800031c0 f   libredefclass030.obj
 0001:000021e0       nsk_ltrace                 00000001800031e0 f   libredefclass030.obj
 0001:00002200       nsk_lvcomplain             0000000180003200 f   libredefclass030.obj
 0001:000023b8       nsk_lvdisplay              00000001800033b8 f   libredefclass030.obj
 0001:00002404       nsk_lverify                0000000180003404 f   libredefclass030.obj
 0001:00002460       nsk_lvtrace                0000000180003460 f   libredefclass030.obj
 0001:000024c0       nsk_printf                 00000001800034c0 f   libredefclass030.obj
 0001:000024e8       nsk_vprintf                00000001800034e8 f   libredefclass030.obj
 0001:0000259c       printf                     000000018000359c f i libredefclass030.obj
 0001:00002a9c       __raise_securityfailure    0000000180003a9c f   MSVCRT:gs_report.obj
 0001:00002ad0       __report_gsfailure         0000000180003ad0 f   MSVCRT:gs_report.obj
 0001:00002d10       __GSHandlerCheck           0000000180003d10 f   MSVCRT:gshandler.obj
 0001:00002d30       __GSHandlerCheckCommon     0000000180003d30 f   MSVCRT:gshandler.obj
 0001:00002da0       __security_check_cookie    0000000180003da0 f   MSVCRT:amdsecgs.obj
 0001:000030e0       _DllMainCRTStartup         00000001800040e0 f   MSVCRT:dll_dllmain.obj
 0001:00003120       __scrt_acquire_startup_lock 0000000180004120 f   MSVCRT:utility.obj
 0001:0000315c       __scrt_dllmain_after_initialize_c 000000018000415c f   MSVCRT:utility.obj
 0001:00003190       __scrt_dllmain_before_initialize_c 0000000180004190 f   MSVCRT:utility.obj
 0001:000031a8       __scrt_dllmain_crt_thread_attach 00000001800041a8 f   MSVCRT:utility.obj
 0001:000031d0       __scrt_dllmain_crt_thread_detach 00000001800041d0 f   MSVCRT:utility.obj
 0001:000031e8       __scrt_dllmain_exception_filter 00000001800041e8 f   MSVCRT:utility.obj
 0001:00003248       __scrt_dllmain_uninitialize_c 0000000180004248 f   MSVCRT:utility.obj
 0001:00003278       __scrt_dllmain_uninitialize_critical 0000000180004278 f   MSVCRT:utility.obj
 0001:0000328c       __scrt_initialize_crt      000000018000428c f   MSVCRT:utility.obj
 0001:000032d8       __scrt_initialize_onexit_tables 00000001800042d8 f   MSVCRT:utility.obj
 0001:00003364       __scrt_is_nonwritable_in_current_image 0000000180004364 f   MSVCRT:utility.obj
 0001:000033fc       __scrt_release_startup_lock 00000001800043fc f   MSVCRT:utility.obj
 0001:00003420       __scrt_uninitialize_crt    0000000180004420 f   MSVCRT:utility.obj
 0001:0000344c       _onexit                    000000018000444c f   MSVCRT:utility.obj
 0001:00003488       atexit                     0000000180004488 f   MSVCRT:utility.obj
 0001:000034a0       __crt_debugger_hook        00000001800044a0 f   MSVCRT:utility_desktop.obj
 0001:000034a8       __scrt_fastfail            00000001800044a8 f   MSVCRT:utility_desktop.obj
 0001:000035f4       _guard_check_icall_nop     00000001800045f4 f i MSVCRT:guard_support.obj
 0001:000035f8       __security_init_cookie     00000001800045f8 f   MSVCRT:gs_support.obj
 0001:000036a4       DllMain                    00000001800046a4 f   MSVCRT:dll_dllmain_stub.obj
 0001:000036c8       ?__scrt_initialize_type_info@@YAXXZ 00000001800046c8 f   MSVCRT:tncleanup.obj
 0001:000036d8       ?__scrt_uninitialize_type_info@@YAXXZ 00000001800046d8 f   MSVCRT:tncleanup.obj
 0001:000036e4       __local_stdio_scanf_options 00000001800046e4 f i MSVCRT:default_local_stdio_options.obj
 0001:000036ec       __scrt_initialize_default_local_stdio_options 00000001800046ec f   MSVCRT:default_local_stdio_options.obj
 0001:00003708       __scrt_get_dyn_tls_init_callback 0000000180004708 f   MSVCRT:dyn_tls_init.obj
 0001:00003710       _RTC_Initialize            0000000180004710 f   MSVCRT:initsect.obj
 0001:0000374c       _RTC_Terminate             000000018000474c f   MSVCRT:initsect.obj
 0001:00003788       __isa_available_init       0000000180004788 f   MSVCRT:cpu_disp.obj
 0001:00003934       _get_startup_argv_mode     0000000180004934 f   MSVCRT:argv_mode.obj
 0001:0000393c       __scrt_is_ucrt_dll_in_use  000000018000493c f   MSVCRT:ucrt_detection.obj
 0001:00003950       memcpy                     0000000180004950 f   vcruntime:VCRUNTIME140.dll
 0001:00003956       memset                     0000000180004956 f   vcruntime:VCRUNTIME140.dll
 0001:0000395c       strchr                     000000018000495c f   vcruntime:VCRUNTIME140.dll
 0001:00003962       __C_specific_handler       0000000180004962 f   vcruntime:VCRUNTIME140.dll
 0001:00003968       __std_type_info_destroy_list 0000000180004968 f   vcruntime:VCRUNTIME140.dll
 0001:0000396e       strcmp                     000000018000496e f   ucrt:api-ms-win-crt-string-l1-1-0.dll
 0001:00003974       strlen                     0000000180004974 f   ucrt:api-ms-win-crt-string-l1-1-0.dll
 0001:0000397a       _initterm                  000000018000497a f   ucrt:api-ms-win-crt-runtime-l1-1-0.dll
 0001:00003980       _initterm_e                0000000180004980 f   ucrt:api-ms-win-crt-runtime-l1-1-0.dll
 0001:00003986       _seh_filter_dll            0000000180004986 f   ucrt:api-ms-win-crt-runtime-l1-1-0.dll
 0001:0000398c       _configure_narrow_argv     000000018000498c f   ucrt:api-ms-win-crt-runtime-l1-1-0.dll
 0001:00003992       _initialize_narrow_environment 0000000180004992 f   ucrt:api-ms-win-crt-runtime-l1-1-0.dll
 0001:00003998       _initialize_onexit_table   0000000180004998 f   ucrt:api-ms-win-crt-runtime-l1-1-0.dll
 0001:0000399e       _register_onexit_function  000000018000499e f   ucrt:api-ms-win-crt-runtime-l1-1-0.dll
 0001:000039a4       _execute_onexit_table      00000001800049a4 f   ucrt:api-ms-win-crt-runtime-l1-1-0.dll
 0001:000039aa       _crt_atexit                00000001800049aa f   ucrt:api-ms-win-crt-runtime-l1-1-0.dll
 0001:000039b0       _cexit                     00000001800049b0 f   ucrt:api-ms-win-crt-runtime-l1-1-0.dll
 0001:000039b8       __acrt_initialize          00000001800049b8 f   MSVCRT:ucrt_stubs.obj
 0001:000039b8       __acrt_thread_attach       00000001800049b8 f   MSVCRT:ucrt_stubs.obj
 0001:000039b8       __acrt_thread_detach       00000001800049b8 f   MSVCRT:ucrt_stubs.obj
 0001:000039b8       __acrt_uninitialize        00000001800049b8 f   MSVCRT:ucrt_stubs.obj
 0001:000039b8       __acrt_uninitialize_critical 00000001800049b8 f   MSVCRT:ucrt_stubs.obj
 0001:000039b8       __scrt_stub_for_acrt_initialize 00000001800049b8 f   MSVCRT:ucrt_stubs.obj
 0001:000039b8       __scrt_stub_for_acrt_thread_attach 00000001800049b8 f   MSVCRT:ucrt_stubs.obj
 0001:000039b8       __scrt_stub_for_acrt_thread_detach 00000001800049b8 f   MSVCRT:ucrt_stubs.obj
 0001:000039b8       __scrt_stub_for_acrt_uninitialize 00000001800049b8 f   MSVCRT:ucrt_stubs.obj
 0001:000039b8       __scrt_stub_for_acrt_uninitialize_critical 00000001800049b8 f   MSVCRT:ucrt_stubs.obj
 0001:000039b8       __vcrt_initialize          00000001800049b8 f   MSVCRT:ucrt_stubs.obj
 0001:000039b8       __vcrt_thread_attach       00000001800049b8 f   MSVCRT:ucrt_stubs.obj
 0001:000039b8       __vcrt_thread_detach       00000001800049b8 f   MSVCRT:ucrt_stubs.obj
 0001:000039b8       __vcrt_uninitialize        00000001800049b8 f   MSVCRT:ucrt_stubs.obj
 0001:000039b8       __vcrt_uninitialize_critical 00000001800049b8 f   MSVCRT:ucrt_stubs.obj
 0001:000039bc       __scrt_stub_for_is_c_termination_complete 00000001800049bc f   MSVCRT:ucrt_stubs.obj
 0001:000039bc       _is_c_termination_complete 00000001800049bc f   MSVCRT:ucrt_stubs.obj
 0001:000039d0       _guard_dispatch_icall_nop  00000001800049d0 f   MSVCRT:guard_dispatch.obj
 0001:000039f0       _guard_xfg_dispatch_icall_nop 00000001800049f0 f   MSVCRT:guard_xfg_dispatch.obj
 0002:00000000       __imp_Sleep                0000000180005000     kernel32:KERNEL32.dll
 0002:00000008       __imp_RtlCaptureContext    0000000180005008     kernel32:KERNEL32.dll
 0002:00000010       __imp_RtlLookupFunctionEntry 0000000180005010     kernel32:KERNEL32.dll
 0002:00000018       __imp_RtlVirtualUnwind     0000000180005018     kernel32:KERNEL32.dll
 0002:00000020       __imp_UnhandledExceptionFilter 0000000180005020     kernel32:KERNEL32.dll
 0002:00000028       __imp_SetUnhandledExceptionFilter 0000000180005028     kernel32:KERNEL32.dll
 0002:00000030       __imp_GetCurrentProcess    0000000180005030     kernel32:KERNEL32.dll
 0002:00000038       __imp_TerminateProcess     0000000180005038     kernel32:KERNEL32.dll
 0002:00000040       __imp_IsProcessorFeaturePresent 0000000180005040     kernel32:KERNEL32.dll
 0002:00000048       __imp_CloseHandle          0000000180005048     kernel32:KERNEL32.dll
 0002:00000050       __imp_InitializeCriticalSectionAndSpinCount 0000000180005050     kernel32:KERNEL32.dll
 0002:00000058       __imp_DeleteCriticalSection 0000000180005058     kernel32:KERNEL32.dll
 0002:00000060       __imp_CreateEventW         0000000180005060     kernel32:KERNEL32.dll
 0002:00000068       __imp_GetModuleHandleW     0000000180005068     kernel32:KERNEL32.dll
 0002:00000070       __imp_GetProcAddress       0000000180005070     kernel32:KERNEL32.dll
 0002:00000078       __imp_IsDebuggerPresent    0000000180005078     kernel32:KERNEL32.dll
 0002:00000080       __imp_QueryPerformanceCounter 0000000180005080     kernel32:KERNEL32.dll
 0002:00000088       __imp_GetCurrentProcessId  0000000180005088     kernel32:KERNEL32.dll
 0002:00000090       __imp_GetCurrentThreadId   0000000180005090     kernel32:KERNEL32.dll
 0002:00000098       __imp_GetSystemTimeAsFileTime 0000000180005098     kernel32:KERNEL32.dll
 0002:000000a0       __imp_DisableThreadLibraryCalls 00000001800050a0     kernel32:KERNEL32.dll
 0002:000000a8       __imp_InitializeSListHead  00000001800050a8     kernel32:KERNEL32.dll
 0002:000000b0       \177KERNEL32_NULL_THUNK_DATA 00000001800050b0     kernel32:KERNEL32.dll
 0002:000000b8       __imp_memcpy               00000001800050b8     vcruntime:VCRUNTIME140.dll
 0002:000000c0       __imp_memset               00000001800050c0     vcruntime:VCRUNTIME140.dll
 0002:000000c8       __imp_strchr               00000001800050c8     vcruntime:VCRUNTIME140.dll
 0002:000000d0       __imp___C_specific_handler 00000001800050d0     vcruntime:VCRUNTIME140.dll
 0002:000000d8       __imp___std_type_info_destroy_list 00000001800050d8     vcruntime:VCRUNTIME140.dll
 0002:000000e0       \177VCRUNTIME140_NULL_THUNK_DATA 00000001800050e0     vcruntime:VCRUNTIME140.dll
 0002:000000e8       __imp_strtol               00000001800050e8     ucrt:api-ms-win-crt-convert-l1-1-0.dll
 0002:000000f0       \177api-ms-win-crt-convert-l1-1-0_NULL_THUNK_DATA 00000001800050f0     ucrt:api-ms-win-crt-convert-l1-1-0.dll
 0002:000000f8       __imp_malloc               00000001800050f8     ucrt:api-ms-win-crt-heap-l1-1-0.dll
 0002:00000100       __imp_free                 0000000180005100     ucrt:api-ms-win-crt-heap-l1-1-0.dll
 0002:00000108       \177api-ms-win-crt-heap-l1-1-0_NULL_THUNK_DATA 0000000180005108     ucrt:api-ms-win-crt-heap-l1-1-0.dll
 0002:00000110       __imp__errno               0000000180005110     ucrt:api-ms-win-crt-runtime-l1-1-0.dll
 0002:00000118       __imp_exit                 0000000180005118     ucrt:api-ms-win-crt-runtime-l1-1-0.dll
 0002:00000120       __imp__cexit               0000000180005120     ucrt:api-ms-win-crt-runtime-l1-1-0.dll
 0002:00000128       __imp__crt_atexit          0000000180005128     ucrt:api-ms-win-crt-runtime-l1-1-0.dll
 0002:00000130       __imp__execute_onexit_table 0000000180005130     ucrt:api-ms-win-crt-runtime-l1-1-0.dll
 0002:00000138       __imp__register_onexit_function 0000000180005138     ucrt:api-ms-win-crt-runtime-l1-1-0.dll
 0002:00000140       __imp__initialize_onexit_table 0000000180005140     ucrt:api-ms-win-crt-runtime-l1-1-0.dll
 0002:00000148       __imp__initialize_narrow_environment 0000000180005148     ucrt:api-ms-win-crt-runtime-l1-1-0.dll
 0002:00000150       __imp__configure_narrow_argv 0000000180005150     ucrt:api-ms-win-crt-runtime-l1-1-0.dll
 0002:00000158       __imp__seh_filter_dll      0000000180005158     ucrt:api-ms-win-crt-runtime-l1-1-0.dll
 0002:00000160       __imp__initterm_e          0000000180005160     ucrt:api-ms-win-crt-runtime-l1-1-0.dll
 0002:00000168       __imp__initterm            0000000180005168     ucrt:api-ms-win-crt-runtime-l1-1-0.dll
 0002:00000170       \177api-ms-win-crt-runtime-l1-1-0_NULL_THUNK_DATA 0000000180005170     ucrt:api-ms-win-crt-runtime-l1-1-0.dll
 0002:00000178       __imp___acrt_iob_func      0000000180005178     ucrt:api-ms-win-crt-stdio-l1-1-0.dll
 0002:00000180       __imp_fflush               0000000180005180     ucrt:api-ms-win-crt-stdio-l1-1-0.dll
 0002:00000188       __imp___stdio_common_vsprintf 0000000180005188     ucrt:api-ms-win-crt-stdio-l1-1-0.dll
 0002:00000190       __imp___stdio_common_vfprintf 0000000180005190     ucrt:api-ms-win-crt-stdio-l1-1-0.dll
 0002:00000198       \177api-ms-win-crt-stdio-l1-1-0_NULL_THUNK_DATA 0000000180005198     ucrt:api-ms-win-crt-stdio-l1-1-0.dll
 0002:000001a0       __imp_strcmp               00000001800051a0     ucrt:api-ms-win-crt-string-l1-1-0.dll
 0002:000001a8       __imp__strdup              00000001800051a8     ucrt:api-ms-win-crt-string-l1-1-0.dll
 0002:000001a8       __imp_strdup               00000001800051a8     ucrt:api-ms-win-crt-string-l1-1-0.dll
 0002:000001b0       __imp_strlen               00000001800051b0     ucrt:api-ms-win-crt-string-l1-1-0.dll
 0002:000001b8       __imp_strpbrk              00000001800051b8     ucrt:api-ms-win-crt-string-l1-1-0.dll
 0002:000001c0       __imp_strncpy              00000001800051c0     ucrt:api-ms-win-crt-string-l1-1-0.dll
 0002:000001c8       \177api-ms-win-crt-string-l1-1-0_NULL_THUNK_DATA 00000001800051c8     ucrt:api-ms-win-crt-string-l1-1-0.dll
 0002:000001d0       __guard_check_icall_fptr   00000001800051d0     MSVCRT:guard_support.obj
 0002:000001d8       __guard_xfg_check_icall_fptr 00000001800051d8     MSVCRT:guard_support.obj
 0002:000001e0       __guard_dispatch_icall_fptr 00000001800051e0     MSVCRT:guard_support.obj
 0002:000001e8       __guard_xfg_dispatch_icall_fptr 00000001800051e8     MSVCRT:guard_support.obj
 0002:000001f0       __guard_xfg_table_dispatch_icall_fptr 00000001800051f0     MSVCRT:guard_support.obj
 0002:000001f8       __castguard_check_failure_os_handled_fptr 00000001800051f8     MSVCRT:guard_support.obj
 0002:00000200       __guard_memcpy_fptr        0000000180005200     vcruntime:softmemtag.obj
 0002:00000208       __xc_a                     0000000180005208     MSVCRT:initializers.obj
 0002:00000210       __xc_z                     0000000180005210     MSVCRT:initializers.obj
 0002:00000218       __xi_a                     0000000180005218     MSVCRT:initializers.obj
 0002:00000228       __xi_z                     0000000180005228     MSVCRT:initializers.obj
 0002:00000230       __xl_a                     0000000180005230     MSVCRT:tlssup.obj
 0002:00000238       __xl_z                     0000000180005238     MSVCRT:tlssup.obj
 0002:00000240       __xp_a                     0000000180005240     MSVCRT:initializers.obj
 0002:00000248       __xp_z                     0000000180005248     MSVCRT:initializers.obj
 0002:00000250       __xt_a                     0000000180005250     MSVCRT:initializers.obj
 0002:00000258       __xt_z                     0000000180005258     MSVCRT:initializers.obj
 0002:00000260       g_refKindStr               0000000180005260     libredefclass030.obj
 0002:00000410       ??_C@_09BPLDFGCI@unknown_0@ 0000000180005410     libredefclass030.obj
 0002:00000420       ??_C@_0BL@FPNMECJD@JVMTI_HEAP_REFERENCE_CLASS@ 0000000180005420     libredefclass030.obj
 0002:00000440       ??_C@_0BL@FKGKKLNM@JVMTI_HEAP_REFERENCE_FIELD@ 0000000180005440     libredefclass030.obj
 0002:00000460       ??_C@_0CD@CAEHCFJF@JVMTI_HEAP_REFERENCE_ARRAY_ELEM@ 0000000180005460     libredefclass030.obj
 0002:00000488       ??_C@_0CC@DNEBMCNK@JVMTI_HEAP_REFERENCE_CLASS_LOAD@ 0000000180005488     libredefclass030.obj
 0002:000004b0       ??_C@_0BN@CJMIPEBB@JVMTI_HEAP_REFERENCE_SIGNERS@ 00000001800054b0     libredefclass030.obj
 0002:000004d0       ??_C@_0CH@HBOIDPEB@JVMTI_HEAP_REFERENCE_PROTECTION@ 00000001800054d0     libredefclass030.obj
 0002:000004f8       ??_C@_0BP@MDKGDGKL@JVMTI_HEAP_REFERENCE_INTERFACE@ 00000001800054f8     libredefclass030.obj
 0002:00000518       ??_C@_0CC@JJMIHNJH@JVMTI_HEAP_REFERENCE_STATIC_FIE@ 0000000180005518     libredefclass030.obj
 0002:00000540       ??_C@_0CD@IDHEEGID@JVMTI_HEAP_REFERENCE_CONSTANT_P@ 0000000180005540     libredefclass030.obj
 0002:00000568       ??_C@_0CA@EFFCHNG@JVMTI_HEAP_REFERENCE_SUPERCLASS@ 0000000180005568     libredefclass030.obj
 0002:00000588       ??_C@_0L@PCDFHGCJ@unknown_11@ 0000000180005588     libredefclass030.obj
 0002:00000598       ??_C@_0L@NJBICFOK@unknown_12@ 0000000180005598     libredefclass030.obj
 0002:000005a8       ??_C@_0L@MAADBEKL@unknown_13@ 00000001800055a8     libredefclass030.obj
 0002:000005b8       ??_C@_0L@IPECICGM@unknown_14@ 00000001800055b8     libredefclass030.obj
 0002:000005c8       ??_C@_0L@JGFJLDCN@unknown_15@ 00000001800055c8     libredefclass030.obj
 0002:000005d8       ??_C@_0L@LNHEOAOO@unknown_16@ 00000001800055d8     libredefclass030.obj
 0002:000005e8       ??_C@_0L@KEGPNBKP@unknown_17@ 00000001800055e8     libredefclass030.obj
 0002:000005f8       ??_C@_0L@CDPHMNGA@unknown_18@ 00000001800055f8     libredefclass030.obj
 0002:00000608       ??_C@_0L@DKOMPMCB@unknown_19@ 0000000180005608     libredefclass030.obj
 0002:00000618       ??_C@_0L@OJGIPJDB@unknown_20@ 0000000180005618     libredefclass030.obj
 0002:00000628       ??_C@_0CA@KAOFNDEM@JVMTI_HEAP_REFERENCE_JNI_GLOBAL@ 0000000180005628     libredefclass030.obj
 0002:00000648       ??_C@_0CC@HPFAJBK@JVMTI_HEAP_REFERENCE_SYSTEM_CLA@ 0000000180005648     libredefclass030.obj
 0002:00000670       ??_C@_0BN@FDEGFOHC@JVMTI_HEAP_REFERENCE_MONITOR@ 0000000180005670     libredefclass030.obj
 0002:00000690       ??_C@_0CB@HKIBCMAJ@JVMTI_HEAP_REFERENCE_STACK_LOCA@ 0000000180005690     libredefclass030.obj
 0002:000006b8       ??_C@_0BP@EAACMMOE@JVMTI_HEAP_REFERENCE_JNI_LOCAL@ 00000001800056b8     libredefclass030.obj
 0002:000006d8       ??_C@_0BM@IJDEOGOE@JVMTI_HEAP_REFERENCE_THREAD@ 00000001800056d8     libredefclass030.obj
 0002:000006f8       ??_C@_0BL@EDGPPKC@JVMTI_HEAP_REFERENCE_OTHER@ 00000001800056f8     libredefclass030.obj
 0002:00000714       ??_C@_04BCJPDBDA@Code@     0000000180005714     libredefclass030.obj
 0002:00000720       ??_C@_0BA@OCLMCFKC@LineNumberTable@ 0000000180005720     libredefclass030.obj
 0002:00000730       ??_C@_0BD@CPAEPILC@LocalVariableTable@ 0000000180005730     libredefclass030.obj
 0002:00000748       ??_C@_0BH@NMBDNHBD@LocalVariableTypeTable@ 0000000180005748     libredefclass030.obj
 0002:00000760       ??_C@_0O@HIHEEDNJ@StackMapTable@ 0000000180005760     libredefclass030.obj
 0002:00000770       ??_C@_0BH@LGECPFHM@redefclass030HotMethod@ 0000000180005770     libredefclass030.obj
 0002:00000788       ??_C@_04PFANPMCN@?$CII?$CJV@ 0000000180005788     libredefclass030.obj
 0002:00000790       ??_C@_0L@HCDIAMJG@?9?5?$CFs?0?5?$CFd?3?5@ 0000000180005790     libredefclass030.obj
 0002:000007a0       ??_C@_0JI@HLPECLFI@?$CD?5?4?4?4?6?$CD?5ERROR?3?5too?5many?5complai@ 00000001800057a0     libredefclass030.obj
 0002:00000840       ??_C@_0ED@JNEKCCOB@The?5following?5fake?5exception?5st@ 0000000180005840     libredefclass030.obj
 0002:00000888       ??_C@_0CN@FCNMDFBH@nsk?4share?4Fake_Exception_for_RU@ 0000000180005888     libredefclass030.obj
 0002:000008b8       ??_C@_08PGFFNAEI@?$CI?$CFs?3?$CFd?$CJ?5@ 00000001800058b8     libredefclass030.obj
 0002:000008c8       ??_C@_0DP@IENMAEGI@s?2test?2hotspot?2jtreg?2vmTestbase@ 00000001800058c8     libredefclass030.obj
 0002:00000908       ??_C@_0BL@NDJLFFJB@?7at?5nsk_lvcomplain?$CI?$CFs?3?$CFd?$CJ?6@ 0000000180005908     libredefclass030.obj
 0002:00000928       ??_C@_0BC@JOOKAFKF@?$CD?5ERROR?3?5?$CFs?0?5?$CFd?3?5@ 0000000180005928     libredefclass030.obj
 0002:00000940       ??_C@_09KJEAHMEH@?$CD?5ERROR?3?5@ 0000000180005940     libredefclass030.obj
 0002:0000094c       ??_C@_02GPIOPFAK@?$DO?$DO@ 000000018000594c     libredefclass030.obj
 0002:00000950       ??_C@_02FODMEDOG@?$DM?$DM@ 0000000180005950     libredefclass030.obj
 0002:00000954       ??_C@_02DJGKEECL@?4?4@     0000000180005954     libredefclass030.obj
 0002:00000958       ??_C@_0O@CJPGJOAF@?9?5?$CFs?0?5?$CFd?3?5?$CFs?5@ 0000000180005958     libredefclass030.obj
 0002:00000968       ??_C@_0CB@IAKPDOIC@?$CD?5?5?5verified?5assertion?5is?5FALSE@ 0000000180005968     libredefclass030.obj
 0002:00000990       ??_C@_0CO@LGONDEPD@stdout?3?5fflush?5failed?5?9?5err?$DN?$CFd?5@ 0000000180005990     libredefclass030.obj
 0002:000009c0       ??_C@_0CO@KBGKJPBD@stderr?3?5fflush?5failed?5?9?5err?$DN?$CFd?5@ 00000001800059c0     libredefclass030.obj
 0002:000009f0       ??_C@_0BB@JCNMKLLK@JVMTI_ERROR_NONE@ 00000001800059f0     libredefclass030.obj
 0002:00000a08       ??_C@_0BL@LDIMKLPH@JVMTI_ERROR_INVALID_THREAD@ 0000000180005a08     libredefclass030.obj
 0002:00000a28       ??_C@_0CB@PJFPAIKJ@JVMTI_ERROR_INVALID_THREAD_GROU@ 0000000180005a28     libredefclass030.obj
 0002:00000a50       ??_C@_0BN@LLMKHMNF@JVMTI_ERROR_INVALID_PRIORITY@ 0000000180005a50     libredefclass030.obj
 0002:00000a70       ??_C@_0CB@MBOFKAGB@JVMTI_ERROR_THREAD_NOT_SUSPENDE@ 0000000180005a70     libredefclass030.obj
 0002:00000a98       ??_C@_0BN@FABOLPBI@JVMTI_ERROR_THREAD_SUSPENDED@ 0000000180005a98     libredefclass030.obj
 0002:00000ab8       ??_C@_0BN@FDGNOBJM@JVMTI_ERROR_THREAD_NOT_ALIVE@ 0000000180005ab8     libredefclass030.obj
 0002:00000ad8       ??_C@_0BL@GOBIFKNJ@JVMTI_ERROR_INVALID_OBJECT@ 0000000180005ad8     libredefclass030.obj
 0002:00000af8       ??_C@_0BK@FCMAJPPC@JVMTI_ERROR_INVALID_CLASS@ 0000000180005af8     libredefclass030.obj
 0002:00000b18       ??_C@_0BP@IKLLBKEB@JVMTI_ERROR_CLASS_NOT_PREPARED@ 0000000180005b18     libredefclass030.obj
 0002:00000b38       ??_C@_0BN@KLPPLKG@JVMTI_ERROR_INVALID_METHODID@ 0000000180005b38     libredefclass030.obj
 0002:00000b58       ??_C@_0BN@BCEKOKND@JVMTI_ERROR_INVALID_LOCATION@ 0000000180005b58     libredefclass030.obj
 0002:00000b78       ??_C@_0BM@DFDGPME@JVMTI_ERROR_INVALID_FIELDID@ 0000000180005b78     libredefclass030.obj
 0002:00000b98       ??_C@_0BL@NELIEPEC@JVMTI_ERROR_NO_MORE_FRAMES@ 0000000180005b98     libredefclass030.obj
 0002:00000bb8       ??_C@_0BJ@BDBECFDM@JVMTI_ERROR_OPAQUE_FRAME@ 0000000180005bb8     libredefclass030.obj
 0002:00000bd8       ??_C@_0BK@MIIFNLOB@JVMTI_ERROR_TYPE_MISMATCH@ 0000000180005bd8     libredefclass030.obj
 0002:00000bf8       ??_C@_0BJ@HPCAOILC@JVMTI_ERROR_INVALID_SLOT@ 0000000180005bf8     libredefclass030.obj
 0002:00000c18       ??_C@_0BG@CHILOPNI@JVMTI_ERROR_DUPLICATE@ 0000000180005c18     libredefclass030.obj
 0002:00000c30       ??_C@_0BG@DIEMLHKM@JVMTI_ERROR_NOT_FOUND@ 0000000180005c30     libredefclass030.obj
 0002:00000c48       ??_C@_0BM@NHMCKHOB@JVMTI_ERROR_INVALID_MONITOR@ 0000000180005c48     libredefclass030.obj
 0002:00000c68       ??_C@_0BO@PPEDAJGL@JVMTI_ERROR_NOT_MONITOR_OWNER@ 0000000180005c68     libredefclass030.obj
 0002:00000c88       ??_C@_0BG@FCAIPEID@JVMTI_ERROR_INTERRUPT@ 0000000180005c88     libredefclass030.obj
 0002:00000ca0       ??_C@_0CB@EGDBNKOI@JVMTI_ERROR_INVALID_CLASS_FORMA@ 0000000180005ca0     libredefclass030.obj
 0002:00000cc8       ??_C@_0CG@DGKOGIAL@JVMTI_ERROR_CIRCULAR_CLASS_DEFI@ 0000000180005cc8     libredefclass030.obj
 0002:00000cf0       ??_C@_0BP@ICEALPKC@JVMTI_ERROR_FAILS_VERIFICATION@ 0000000180005cf0     libredefclass030.obj
 0002:00000d10       ??_C@_0DC@JDACLMIO@JVMTI_ERROR_UNSUPPORTED_REDEFIN@ 0000000180005d10     libredefclass030.obj
 0002:00000d48       ??_C@_0DE@GKDKNOMJ@JVMTI_ERROR_UNSUPPORTED_REDEFIN@ 0000000180005d48     libredefclass030.obj
 0002:00000d80       ??_C@_0BO@LAFKIOG@JVMTI_ERROR_INVALID_TYPESTATE@ 0000000180005d80     libredefclass030.obj
 0002:00000da0       ??_C@_0DH@INDGCLLB@JVMTI_ERROR_UNSUPPORTED_REDEFIN@ 0000000180005da0     libredefclass030.obj
 0002:00000dd8       ??_C@_0DE@NHEOMMGI@JVMTI_ERROR_UNSUPPORTED_REDEFIN@ 0000000180005dd8     libredefclass030.obj
 0002:00000e10       ??_C@_0CA@EKPNJOEP@JVMTI_ERROR_UNSUPPORTED_VERSION@ 0000000180005e10     libredefclass030.obj
 0002:00000e30       ??_C@_0BN@OFFMAHHL@JVMTI_ERROR_NAMES_DONT_MATCH@ 0000000180005e30     libredefclass030.obj
 0002:00000e50       ??_C@_0DN@HHBBLAKE@JVMTI_ERROR_UNSUPPORTED_REDEFIN@ 0000000180005e50     libredefclass030.obj
 0002:00000e90       ??_C@_0DO@HMBGBGNA@JVMTI_ERROR_UNSUPPORTED_REDEFIN@ 0000000180005e90     libredefclass030.obj
 0002:00000ed0       ??_C@_0BP@PBECGKHJ@JVMTI_ERROR_UNMODIFIABLE_CLASS@ 0000000180005ed0     libredefclass030.obj
 0002:00000ef0       ??_C@_0BK@CANILEHF@JVMTI_ERROR_NOT_AVAILABLE@ 0000000180005ef0     libredefclass030.obj
 0002:00000f10       ??_C@_0CE@INJKMEFK@JVMTI_ERROR_MUST_POSSESS_CAPABI@ 0000000180005f10     libredefclass030.obj
 0002:00000f38       ??_C@_0BJ@LBFPFPDM@JVMTI_ERROR_NULL_POINTER@ 0000000180005f38     libredefclass030.obj
 0002:00000f58       ??_C@_0BP@CHJPNNEM@JVMTI_ERROR_ABSENT_INFORMATION@ 0000000180005f58     libredefclass030.obj
 0002:00000f78       ??_C@_0BP@OMFMNLC@JVMTI_ERROR_INVALID_EVENT_TYPE@ 0000000180005f78     libredefclass030.obj
 0002:00000f98       ??_C@_0BN@BIBNPHHO@JVMTI_ERROR_ILLEGAL_ARGUMENT@ 0000000180005f98     libredefclass030.obj
 0002:00000fb8       ??_C@_0BK@KKNDHDCE@JVMTI_ERROR_NATIVE_METHOD@ 0000000180005fb8     libredefclass030.obj
 0002:00000fd8       ??_C@_0BK@PMKCFHAE@JVMTI_ERROR_OUT_OF_MEMORY@ 0000000180005fd8     libredefclass030.obj
 0002:00000ff8       ??_C@_0BK@NNJBDMNB@JVMTI_ERROR_ACCESS_DENIED@ 0000000180005ff8     libredefclass030.obj
 0002:00001018       ??_C@_0BI@GHECLMNC@JVMTI_ERROR_WRONG_PHASE@ 0000000180006018     libredefclass030.obj
 0002:00001030       ??_C@_0BF@OLIHJOII@JVMTI_ERROR_INTERNAL@ 0000000180006030     libredefclass030.obj
 0002:00001048       ??_C@_0BO@EOHGKJHI@JVMTI_ERROR_UNATTACHED_THREAD@ 0000000180006048     libredefclass030.obj
 0002:00001068       ??_C@_0CA@LKHFDACL@JVMTI_ERROR_INVALID_ENVIRONMENT@ 0000000180006068     libredefclass030.obj
 0002:00001088       ??_C@_0BA@MMFHLOKK@?$DMunknown?5error?$DO@ 0000000180006088     libredefclass030.obj
 0002:00001098       ??_C@_0CF@CBHOKDB@throwable?5?$DN?5jni?9?$DOExceptionOccur@ 0000000180006098     libredefclass030.obj
 0002:000010c0       ??_C@_03OFAPEBGM@?$CFs?6@  00000001800060c0     libredefclass030.obj
 0002:000010c8       ??_C@_0DM@LPIGEGNJ@s?2test?2hotspot?2jtreg?2vmTestbase@ 00000001800060c8     libredefclass030.obj
 0002:00001108       ??_C@_0CC@NFCNPEPK@Exception?5in?5JNI?5call?5?$CIcleared?$CJ@ 0000000180006108     libredefclass030.obj
 0002:00001130       ??_C@_0BJ@IBAKFIKF@jni?9?$DOExceptionDescribe?$CI?$CJ@ 0000000180006130     libredefclass030.obj
 0002:00001150       ??_C@_0BG@GGKALKMH@jni?9?$DOExceptionClear?$CI?$CJ@ 0000000180006150     libredefclass030.obj
 0002:00001168       ??_C@_0CF@JMGFGJLJ@?$CD?5?5?5verified?5JNI?5assertion?5is?5F@ 0000000180006168     libredefclass030.obj
 0002:00001190       ??_C@_07KBAMPNJK@verbose@  0000000180006190     libredefclass030.obj
 0002:00001198       ??_C@_0DN@PKJBOLAP@nsk_jvmti_parseOptions?$CI?$CJ?3?5unexp@ 0000000180006198     libredefclass030.obj
 0002:000011d8       ??_C@_05IMBNNINJ@trace@    00000001800061d8     libredefclass030.obj
 0002:000011e0       ??_C@_0DD@BJKGNDMB@nsk_jvmti_parseOptions?$CI?$CJ?3?5no?5va@ 00000001800061e0     libredefclass030.obj
 0002:00001214       ??_C@_04CGFJFPFD@none@     0000000180006214     libredefclass030.obj
 0002:0000121c       ??_C@_06BMELKFMA@before@   000000018000621c     libredefclass030.obj
 0002:00001224       ??_C@_05CMKPCFDK@after@    0000000180006224     libredefclass030.obj
 0002:0000122c       ??_C@_03NFKEKGGK@all@      000000018000622c     libredefclass030.obj
 0002:00001230       ??_C@_0DM@NDNJGJKE@nsk_jvmti_parseOptions?$CI?$CJ?3?5uexpe@ 0000000180006230     libredefclass030.obj
 0002:00001270       ??_C@_08NBBJKJO@waittime@  0000000180006270     libredefclass030.obj
 0002:00001280       ??_C@_0DO@CMHGAOHC@nsk_jvmti_parseOptions?$CI?$CJ?3?5not?5i@ 0000000180006280     libredefclass030.obj
 0002:000012c0       ??_C@_0DL@LNMPBDLN@nsk_jvmti_parseOptions?$CI?$CJ?3?5negat@ 00000001800062c0     libredefclass030.obj
 0002:00001300       ??_C@_0DA@GMFJNOJH@nsk_jvmti_parseOptions?$CI?$CJ?3?5unkno@ 0000000180006300     libredefclass030.obj
 0002:00001330       ??_C@_0CO@CCIAMEAN@nsk_jvmti_parseOptions?$CI?$CJ?3?5found@ 0000000180006330     libredefclass030.obj
 0002:00001360       ??_C@_0CJ@OEGPCGDL@nsk_jvmti_parseOptions?$CI?$CJ?3?5out?5o@ 0000000180006360     libredefclass030.obj
 0002:00001390       ??_C@_0DI@NMBHPGGF@nsk_jvmti_parseOptions?$CI?$CJ?3?5too?5m@ 0000000180006390     libredefclass030.obj
 0002:000013c8       ??_C@_03POGCGECB@?5?0?$HO@ 00000001800063c8     libredefclass030.obj
 0002:000013d0       ??_C@_0CB@MLNJNCLJ@?5?5jvmti?5error?3?5code?$DN?$CFd?0?5name?$DN?$CFs@ 00000001800063d0     libredefclass030.obj
 0002:000013f8       ??_C@_0CD@OHBGDKMK@?$CD?5?5?5jvmti?5error?3?5code?$DN?$CFd?0?5name?$DN@ 00000001800063f8     libredefclass030.obj
 0002:00001420       ??_C@_0CG@JNNCGPHB@?$CD?5?5?5error?5expected?3?5code?$DN?$CFd?0?5na@ 0000000180006420     libredefclass030.obj
 0002:00001450       ??_C@_0EB@IMGKPCGE@?$CIstr_obj?5?$DN?5jni?9?$DONewStringUTF?$CIco@ 0000000180006450     libredefclass030.obj
 0002:000014a0       ??_C@_0EA@HFOGGBCC@s?2test?2hotspot?2jtreg?2vmTestbase@ 00000001800064a0     libredefclass030.obj
 0002:000014e0       ??_C@_05KKCIMGE@error@     00000001800064e0     libredefclass030.obj
 0002:000014e8       ??_C@_0BD@HGNAOMCP@agent_data_monitor@ 00000001800064e8     libredefclass030.obj
 0002:00001500       ??_C@_0EB@OGCLGKLN@javaVM?9?$DOGetEnv?$CI?$CIvoid?5?$CK?$CK?$CJ?$CGjvmti_@ 0000000180006500     libredefclass030.obj
 0002:00001550       ??_C@_0EA@PNBCDMOA@s?2test?2hotspot?2jtreg?2vmTestbase@ 0000000180006550     libredefclass030.obj
 0002:00001590       ??_C@_0CI@DDPIFBGM@init_agent_data?$CIjvmti_env?0?5?$CGage@ 0000000180006590     libredefclass030.obj
 0002:000015b8       ??_C@_0DI@ILAHDLMP@?$CI?$CKagentThreadProc?$CJ?$CIjvmti_env?0?5a@ 00000001800065b8     libredefclass030.obj
 0002:000015f0       ??_C@_0BD@KDBALNLB@JVMTI?5agent?5thread@ 00000001800065f0     libredefclass030.obj
 0002:00001608       ??_C@_0BB@NOKBFPFO@java?1lang?1Thread@ 0000000180006608     libredefclass030.obj
 0002:0000161c       ??_C@_06FALKBLGB@?$DMinit?$DO@ 000000018000661c     libredefclass030.obj
 0002:00001628       ??_C@_0BG@IKDDPPGD@?$CILjava?1lang?1String?$DL?$CJV@ 0000000180006628     libredefclass030.obj
 0002:00001640       ??_C@_0EB@IFJBFEKC@?$CIthreadClass?5?$DN?5jni_env?9?$DOFindCla@ 0000000180006640     libredefclass030.obj
 0002:00001690       ??_C@_0GF@FGFIBKKL@?$CIthreadCtor?5?$DN?5jni_env?9?$DOGetMetho@ 0000000180006690     libredefclass030.obj
 0002:000016f8       ??_C@_0DN@NCPDJLOG@?$CIthreadName?5?$DN?5jni_env?9?$DONewStrin@ 00000001800066f8     libredefclass030.obj
 0002:00001740       ??_C@_0FE@PFKODBGC@?$CIthreadObject?5?$DN?5jni_env?9?$DONewObj@ 0000000180006740     libredefclass030.obj
 0002:000017a0       ??_C@_0ED@HOBAHHJI@?$CIthreadGlobalRef?5?$DN?5jni_env?9?$DONew@ 00000001800067a0     libredefclass030.obj
 0002:000017f0       ??_C@_0FN@HNJJAHFC@jvmti_env?9?$DORunAgentThread?$CIagent@ 00000001800067f0     libredefclass030.obj
 0002:00001850       ??_C@_0EA@MOJDNKDF@Debuggee?5status?5sync?5aborted?5be@ 0000000180006850     libredefclass030.obj
 0002:00001890       ??_C@_0CO@PGPGMHBJ@No?5status?5sync?5occured?5for?5time@ 0000000180006890     libredefclass030.obj
 0002:000018c0       ??_C@_0CL@DOEBDPKJ@Debuggee?5was?5not?5suspended?5on?5s@ 00000001800068c0     libredefclass030.obj
 0002:000018f0       ??_C@_0EA@EEOEJAEN@status?5?$DN?5syncDebuggeeStatus?$CIjni@ 00000001800068f0     libredefclass030.obj
 0002:00001930       ??_C@_0BL@JBCFNBMB@nsk_jvmti_resetAgentData?$CI?$CJ@ 0000000180006930     libredefclass030.obj
 0002:00001950       ??_C@_0DN@NNGECJON@jvmti_env?9?$DOSetEventNotification@ 0000000180006950     libredefclass030.obj
 0002:00001990       ??_C@_0EL@LPBEELIP@s?2test?2hotspot?2jtreg?2vmTestbase@ 0000000180006990     libredefclass030.obj
 0002:000019e0       ??_C@_0CK@JDAMFDMJ@jvmti?9?$DOSetTag?$CIo?0?5tag?$CJ?5?$DN?$DN?5JVMTI_@ 00000001800069e0     libredefclass030.obj
 0002:00001a10       ??_C@_0CC@DAMNHKNI@Can?8t?5set?5tag?5?$CFli?5for?5object?5?$CFl@ 0000000180006a10     libredefclass030.obj
 0002:00001a38       ??_C@_0DL@HAJPNKEF@jvmti?9?$DOGetObjectHashCode?$CIo?0?5?$CGha@ 0000000180006a38     libredefclass030.obj
 0002:00001a78       ??_C@_0BL@JFPIEOBF@Can?8t?5get?5hash?5object?5?$CFlx?6@ 0000000180006a78     libredefclass030.obj
 0002:00001a98       ??_C@_0BG@DICPHBKN@setTag?3?5?$CF08x?5?$DM?9?5?$CF?53li@ 0000000180006a98     libredefclass030.obj
 0002:00001ab0       ??_C@_0DH@FCEEBDMJ@?$CIs?5?$DN?5jni?9?$DOGetStringUTFChars?$CIsIn@ 0000000180006ab0     libredefclass030.obj
 0002:00001ae8       ??_C@_0BJ@OKKGHDCN@Can?8t?5get?5string?5at?5?$CF?$CDp?6@ 0000000180006ae8     libredefclass030.obj
 0002:00001b08       ??_C@_0BP@EKFLGGFJ@Can?8t?5get?5string?5at?5?$CF?$CDp?3?5null?6@ 0000000180006b08     libredefclass030.obj
 0002:00001b28       ??_C@_06ICODBHCL@?5?1?1?5?$CFs@ 0000000180006b28     libredefclass030.obj
 0002:00001b30       ??_C@_0DB@KGFPLEGO@?$CIr?5?$DN?5jvmti?9?$DOGetTag?$CIo?0?5?$CGtag?$CJ?$CJ?5?$DN?$DN@ 0000000180006b30     libredefclass030.obj
 0002:00001b68       ??_C@_0CO@PDAGBCGJ@Can?8t?5GetTag?5for?5object?5?$CFlx?4?5Re@ 0000000180006b68     libredefclass030.obj
 0002:00001b98       ??_C@_0CH@HPEODOHC@TEST_BUG?3?5Max?4?5number?5of?5refs?5r@ 0000000180006b98     libredefclass030.obj
 0002:00001bc0       ??_C@_0DI@PHFCABIM@?$CIr?5?$DN?5jvmti?9?$DOGetTag?$CIfrom?0?5?$CGtagFr@ 0000000180006bc0     libredefclass030.obj
 0002:00001bf8       ??_C@_0DI@MDEGFNKD@TEST_BUG?3?5Can?8t?5GetTag?5for?5obje@ 0000000180006bf8     libredefclass030.obj
 0002:00001c30       ??_C@_0DE@MLELJAHM@?$CIr?5?$DN?5jvmti?9?$DOGetTag?$CIto?0?5?$CGtagTo?$CJ?$CJ@ 0000000180006c30     libredefclass030.obj
 0002:00001c68       ??_C@_0CK@EOPGBGKK@isRedefinitionOccurred?5is?5calle@ 0000000180006c68     libredefclass030.obj
 0002:00001ca0       ??_C@_0FK@CDDBJAPO@s?2test?2hotspot?2jtreg?2vmTestbase@ 0000000180006ca0     libredefclass030.obj
 0002:00001d00       ??_C@_0BN@NEEOIPLO@notifyNativeAgent?5is?5called?6@ 0000000180006d00     libredefclass030.obj
 0002:00001d20       ??_C@_0CI@GOIGCOJA@CompiledMethodLoad?5event?5receiv@ 0000000180006d20     libredefclass030.obj
 0002:00001d48       ??_C@_0DH@GCOJDBIO@jvmti_env?9?$DOGetMethodName?$CImethod@ 0000000180006d48     libredefclass030.obj
 0002:00001d80       ??_C@_0ID@FKGELPPN@?7method?3?5name?$DN?$CC?$CFs?$CC?5signature?$DN?$CC?$CF@ 0000000180006d80     libredefclass030.obj
 0002:00001e08       ??_C@_0DD@CIFOBJCN@CompiledMethodLoad?3?5a?5tested?5ho@ 0000000180006e08     libredefclass030.obj
 0002:00001e40       ??_C@_0DI@DJLHKDHD@Compilation?5occured?5before?5meth@ 0000000180006e40     libredefclass030.obj
 0002:00001e78       ??_C@_0CF@NAKKFALD@CompiledMethodUnload?5event?5rece@ 0000000180006e78     libredefclass030.obj
 0002:00001ea0       ??_C@_0DN@NNJMMNHN@for?3?5?7method?3?5name?$DN?$CC?$CFs?$CC?5signatu@ 0000000180006ea0     libredefclass030.obj
 0002:00001ee0       ??_C@_0DM@NNJEKMJH@agentProc?3?5waiting?5for?5the?5debu@ 0000000180006ee0     libredefclass030.obj
 0002:00001f20       ??_C@_0CH@NCEJGEND@agentProc?3?5resuming?5the?5debugge@ 0000000180006f20     libredefclass030.obj
 0002:00001f50       ??_C@_0EB@BIIGAOGH@agentProc?3?5sending?5all?5generate@ 0000000180006f50     libredefclass030.obj
 0002:00001f98       ??_C@_0DI@BFMHPNME@jvmti?9?$DOGenerateEvents?$CIJVMTI_EVE@ 0000000180006f98     libredefclass030.obj
 0002:00001fd0       ??_C@_0DH@DPOOGNHJ@agentProc?3?5waiting?5for?5hotspot?5@ 0000000180006fd0     libredefclass030.obj
 0002:00002010       ??_C@_0GO@BBNMOEDN@WARNING?3?5CompiledMethodLoad?5eve@ 0000000180007010     libredefclass030.obj
 0002:00002080       ??_C@_0CF@BBGBFFAI@agentProc?3?5hotspot?5method?5compi@ 0000000180007080     libredefclass030.obj
 0002:000020a8       ??_C@_0DK@PKJDKBKO@jvmti_env?9?$DOGetMethodDeclaringCl@ 00000001800070a8     libredefclass030.obj
 0002:000020e8       ??_C@_0DK@LDGEOOHJ@jvmti_env?9?$DOGetClassSignature?$CIde@ 00000001800070e8     libredefclass030.obj
 0002:00002128       ??_C@_0DC@NHCDKGHH@agentProc?3?5hotspot?5method?5class@ 0000000180007128     libredefclass030.obj
 0002:00002160       ??_C@_0EI@KJBONIIM@agentProc?3?5?$DO?$DO?$DO?$DO?$DO?$DO?$DO?$DO?5Invoke?5Rede@ 0000000180007160     libredefclass030.obj
 0002:000021a8       ??_C@_0CF@OBOBAJEI@jvmti?9?$DORedefineClasses?$CI1?0?5?$CGclas@ 00000001800071a8     libredefclass030.obj
 0002:000021d0       ??_C@_0DM@OBAGCLFD@agentProc?3?5?$DM?$DM?$DM?$DM?$DM?$DM?$DM?$DM?5RedefineCla@ 00000001800071d0     libredefclass030.obj
 0002:00002210       ??_C@_0DN@KDPOPOJI@agentProc?3?5waiting?5for?5the?5debu@ 0000000180007210     libredefclass030.obj
 0002:00002250       ??_C@_0DA@MJHFJKIM@agentProc?3?5final?5resuming?5of?5th@ 0000000180007250     libredefclass030.obj
 0002:00002280       ??_C@_0BG@FMNKMBB@agentProc?3?5finished?6?6@ 0000000180007280     libredefclass030.obj
 0002:00002298       ??_C@_0CA@MNKGCBCG@nsk_jvmti_parseOptions?$CIoptions?$CJ@ 0000000180007298     libredefclass030.obj
 0002:000022b8       ??_C@_0BD@FAKCJAOH@waittime?$DN?$CFd?5msecs?6@ 00000001800072b8     libredefclass030.obj
 0002:000022d0       ??_C@_0DN@MIAMNFPH@?$CIjvmti?5?$DN?5nsk_jvmti_createJVMTIE@ 00000001800072d0     libredefclass030.obj
 0002:00002310       ??_C@_0BO@DBKDIPGD@jvmti?9?$DOAddCapabilities?$CI?$CGcaps?$CJ@ 0000000180007310     libredefclass030.obj
 0002:00002330       ??_C@_0BN@HGIKGGD@setting?5event?5callbacks?5?4?4?4?6@ 0000000180007330     libredefclass030.obj
 0002:00002350       ??_C@_0DI@NJCFGEGC@jvmti?9?$DOSetEventCallbacks?$CI?$CGcallb@ 0000000180007350     libredefclass030.obj
 0002:00002388       ??_C@_0DC@EEJJNFPC@setting?5event?5callbacks?5done?6en@ 0000000180007388     libredefclass030.obj
 0002:000023c0       ??_C@_0BL@GBOGNFCP@enabling?5the?5events?5done?6?6@ 00000001800073c0     libredefclass030.obj
 0002:000023e0       ??_C@_0CL@PIACJIPK@nsk_jvmti_setAgentProc?$CIagentPro@ 00000001800073e0     libredefclass030.obj
 0002:00002420       ??_C@_1EC@JIJBPKFM@?$AAa?$AAp?$AAi?$AA?9?$AAm?$AAs?$AA?9?$AAw?$AAi?$AAn?$AA?9?$AAc?$AAo?$AAr?$AAe@ 0000000180007420     MSVCRT:thread_safe_statics.obj
 0002:00002468       ??_C@_1BK@MGMFAEKH@?$AAk?$AAe?$AAr?$AAn?$AAe?$AAl?$AA3?$AA2?$AA?4?$AAd?$AAl?$AAl@ 0000000180007468     MSVCRT:thread_safe_statics.obj
 0002:00002488       ??_C@_0BJ@JEBJOJFJ@SleepConditionVariableCS@ 0000000180007488     MSVCRT:thread_safe_statics.obj
 0002:000024a8       ??_C@_0BJ@PGPPEPCC@WakeAllConditionVariable@ 00000001800074a8     MSVCRT:thread_safe_statics.obj
 0002:000024c8       _pDefaultRawDllMain        00000001800074c8     MSVCRT:dll_dllmain.obj
 0002:000024c8       _pRawDllMain               00000001800074c8     MSVCRT:dll_dllmain.obj
 0002:000024d0       __xmm@ffffffffffffffffffffffffffffffff 00000001800074d0     MSVCRT:utility.obj
 0002:000024e0       _load_config_used          00000001800074e0     MSVCRT:loadcfg.obj
 0002:00002700       _tls_used                  0000000180007700     MSVCRT:tlssup.obj
 0002:00002728       __volatile_metadata        0000000180007728     <linker-defined>
 0002:00002b40       __rtc_iaa                  0000000180007b40     MSVCRT:initsect.obj
 0002:00002b48       __rtc_izz                  0000000180007b48     MSVCRT:initsect.obj
 0002:00002b50       __rtc_taa                  0000000180007b50     MSVCRT:initsect.obj
 0002:00002b58       __rtc_tzz                  0000000180007b58     MSVCRT:initsect.obj
 0002:00002b60       _tls_start                 0000000180007b60     MSVCRT:tlssup.obj
 0002:00002b64       _Init_thread_epoch         0000000180007b64     MSVCRT:thread_safe_statics.obj
 0002:00002b68       _tls_end                   0000000180007b68     MSVCRT:tlssup.obj
 0002:00003364       __IMPORT_DESCRIPTOR_KERNEL32 0000000180008364     kernel32:KERNEL32.dll
 0002:00003378       __IMPORT_DESCRIPTOR_VCRUNTIME140 0000000180008378     vcruntime:VCRUNTIME140.dll
 0002:0000338c       __IMPORT_DESCRIPTOR_api-ms-win-crt-heap-l1-1-0 000000018000838c     ucrt:api-ms-win-crt-heap-l1-1-0.dll
 0002:000033a0       __IMPORT_DESCRIPTOR_api-ms-win-crt-runtime-l1-1-0 00000001800083a0     ucrt:api-ms-win-crt-runtime-l1-1-0.dll
 0002:000033b4       __IMPORT_DESCRIPTOR_api-ms-win-crt-convert-l1-1-0 00000001800083b4     ucrt:api-ms-win-crt-convert-l1-1-0.dll
 0002:000033c8       __IMPORT_DESCRIPTOR_api-ms-win-crt-stdio-l1-1-0 00000001800083c8     ucrt:api-ms-win-crt-stdio-l1-1-0.dll
 0002:000033dc       __IMPORT_DESCRIPTOR_api-ms-win-crt-string-l1-1-0 00000001800083dc     ucrt:api-ms-win-crt-string-l1-1-0.dll
 0002:000033f0       __NULL_IMPORT_DESCRIPTOR   00000001800083f0     kernel32:KERNEL32.dll
 0003:00000048       _Init_global_epoch         0000000180009048     MSVCRT:thread_safe_statics.obj
 0003:00000050       __security_cookie          0000000180009050     MSVCRT:gs_cookie.obj
 0003:00000058       __security_cookie_complement 0000000180009058     MSVCRT:gs_cookie.obj
 0003:00000060       __scrt_native_dllmain_reason 0000000180009060     MSVCRT:utility.obj
 0003:00000068       __isa_available            0000000180009068     MSVCRT:cpu_disp.obj
 0003:0000006c       __isa_enabled              000000018000906c     MSVCRT:cpu_disp.obj
 0003:00000070       __memset_fast_string_threshold 0000000180009070     MSVCRT:cpu_disp.obj
 0003:00000078       __memset_nt_threshold      0000000180009078     MSVCRT:cpu_disp.obj
 0003:00000080       __scrt_ucrt_dll_is_in_use  0000000180009080     MSVCRT:ucrt_stubs.obj
 0003:00000090       g_wrongHeapCallbacks       0000000180009090     libredefclass030.obj
 0003:00000110       g_szTagInfo                0000000180009110     libredefclass030.obj
 0003:00002050       g_tagFlags                 000000018000b050     libredefclass030.obj
 0003:00002438       g_refsToVerifyCnt          000000018000b438     libredefclass030.obj
 0003:0000243c       g_fakeUserData             000000018000b43c     libredefclass030.obj
 0003:00002440       g_tagVisitCount            000000018000b440     libredefclass030.obj
 0003:000033e0       g_refsToVerify             000000018000c3e0     libredefclass030.obj
 0003:0001aae0       g_userDataError            0000000180023ae0     libredefclass030.obj
 0003:0001aca0       ?_OptionsStorage@?1??__local_stdio_printf_options@@9@4_KA 0000000180023ca0     libredefclass030.obj
 0003:0001b268       _tls_index                 0000000180024268     MSVCRT:tlssup.obj
 0003:0001b270       __scrt_current_native_startup_state 0000000180024270     MSVCRT:utility.obj
 0003:0001b278       __scrt_native_startup_lock 0000000180024278     MSVCRT:utility.obj
 0003:0001b2b8       __scrt_debugger_hook_flag  00000001800242b8     MSVCRT:utility_desktop.obj
 0003:0001b2c0       ?__type_info_root_node@@3U__type_info_node@@A 00000001800242c0     MSVCRT:tncleanup.obj
 0003:0001b2d0       ?_OptionsStorage@?1??__local_stdio_scanf_options@@9@4_KA 00000001800242d0     MSVCRT:default_local_stdio_options.obj
 0003:0001b2d8       __favor                    00000001800242d8     MSVCRT:cpu_disp.obj
 0003:0001b2e0       __dyn_tls_init_callback    00000001800242e0     <common>

 entry point at        0001:000030e0

 Static symbols

 0000:fffd9000       .debug$S                   0000000180000000     redefclass030.exp
 0000:fffd9000       .debug$S                   0000000180000000     vcruntime:VCRUNTIME140.dll
 0000:fffd9000       .debug$S                   0000000180000000     vcruntime:VCRUNTIME140.dll
 0000:fffd9000       .debug$S                   0000000180000000     vcruntime:VCRUNTIME140.dll
 0000:fffd9000       .debug$S                   0000000180000000     vcruntime:VCRUNTIME140.dll
 0000:fffd9000       .debug$S                   0000000180000000     vcruntime:VCRUNTIME140.dll
 0000:fffd9000       .debug$S                   0000000180000000     vcruntime:VCRUNTIME140.dll
 0000:fffd9000       .debug$S                   0000000180000000     vcruntime:VCRUNTIME140.dll
 0000:fffd9000       .debug$S                   0000000180000000     ucrt:api-ms-win-crt-convert-l1-1-0.dll
 0000:fffd9000       .debug$S                   0000000180000000     ucrt:api-ms-win-crt-heap-l1-1-0.dll
 0000:fffd9000       .debug$S                   0000000180000000     ucrt:api-ms-win-crt-heap-l1-1-0.dll
 0000:fffd9000       .debug$S                   0000000180000000     ucrt:api-ms-win-crt-heap-l1-1-0.dll
 0000:fffd9000       .debug$S                   0000000180000000     ucrt:api-ms-win-crt-heap-l1-1-0.dll
 0000:fffd9000       .debug$S                   0000000180000000     ucrt:api-ms-win-crt-runtime-l1-1-0.dll
 0000:fffd9000       .debug$S                   0000000180000000     ucrt:api-ms-win-crt-runtime-l1-1-0.dll
 0000:fffd9000       .debug$S                   0000000180000000     ucrt:api-ms-win-crt-runtime-l1-1-0.dll
 0000:fffd9000       .debug$S                   0000000180000000     ucrt:api-ms-win-crt-runtime-l1-1-0.dll
 0000:fffd9000       .debug$S                   0000000180000000     ucrt:api-ms-win-crt-runtime-l1-1-0.dll
 0000:fffd9000       .debug$S                   0000000180000000     ucrt:api-ms-win-crt-runtime-l1-1-0.dll
 0000:fffd9000       .debug$S                   0000000180000000     ucrt:api-ms-win-crt-runtime-l1-1-0.dll
 0000:fffd9000       .debug$S                   0000000180000000     ucrt:api-ms-win-crt-runtime-l1-1-0.dll
 0000:fffd9000       .debug$S                   0000000180000000     ucrt:api-ms-win-crt-runtime-l1-1-0.dll
 0000:fffd9000       .debug$S                   0000000180000000     ucrt:api-ms-win-crt-runtime-l1-1-0.dll
 0000:fffd9000       .debug$S                   0000000180000000     ucrt:api-ms-win-crt-runtime-l1-1-0.dll
 0000:fffd9000       .debug$S                   0000000180000000     ucrt:api-ms-win-crt-runtime-l1-1-0.dll
 0000:fffd9000       .debug$S                   0000000180000000     ucrt:api-ms-win-crt-runtime-l1-1-0.dll
 0000:fffd9000       .debug$S                   0000000180000000     ucrt:api-ms-win-crt-runtime-l1-1-0.dll
 0000:fffd9000       .debug$S                   0000000180000000     ucrt:api-ms-win-crt-runtime-l1-1-0.dll
 0000:fffd9000       .debug$S                   0000000180000000     ucrt:api-ms-win-crt-runtime-l1-1-0.dll
 0000:fffd9000       .debug$S                   0000000180000000     ucrt:api-ms-win-crt-stdio-l1-1-0.dll
 0000:fffd9000       .debug$S                   0000000180000000     ucrt:api-ms-win-crt-stdio-l1-1-0.dll
 0000:fffd9000       .debug$S                   0000000180000000     ucrt:api-ms-win-crt-stdio-l1-1-0.dll
 0000:fffd9000       .debug$S                   0000000180000000     ucrt:api-ms-win-crt-stdio-l1-1-0.dll
 0000:fffd9000       .debug$S                   0000000180000000     ucrt:api-ms-win-crt-stdio-l1-1-0.dll
 0000:fffd9000       .debug$S                   0000000180000000     ucrt:api-ms-win-crt-stdio-l1-1-0.dll
 0000:fffd9000       .debug$S                   0000000180000000     ucrt:api-ms-win-crt-stdio-l1-1-0.dll
 0000:fffd9000       .debug$S                   0000000180000000     ucrt:api-ms-win-crt-stdio-l1-1-0.dll
 0000:fffd9000       .debug$S                   0000000180000000     ucrt:api-ms-win-crt-stdio-l1-1-0.dll
 0000:fffd9000       .debug$S                   0000000180000000     ucrt:api-ms-win-crt-stdio-l1-1-0.dll
 0000:fffd9000       .debug$S                   0000000180000000     ucrt:api-ms-win-crt-string-l1-1-0.dll
 0000:fffd9000       .debug$S                   0000000180000000     ucrt:api-ms-win-crt-string-l1-1-0.dll
 0000:fffd9000       .debug$S                   0000000180000000     ucrt:api-ms-win-crt-string-l1-1-0.dll
 0000:fffd9000       .debug$S                   0000000180000000     ucrt:api-ms-win-crt-string-l1-1-0.dll
 0000:fffd9000       .debug$S                   0000000180000000     ucrt:api-ms-win-crt-string-l1-1-0.dll
 0000:fffd9000       .debug$S                   0000000180000000     ucrt:api-ms-win-crt-string-l1-1-0.dll
 0000:fffd9000       .debug$S                   0000000180000000     ucrt:api-ms-win-crt-string-l1-1-0.dll
 0000:fffd9000       .debug$S                   0000000180000000     ucrt:api-ms-win-crt-string-l1-1-0.dll
 0000:fffd9000       .debug$S                   0000000180000000     kernel32:KERNEL32.dll
 0000:fffd9000       .debug$S                   0000000180000000     kernel32:KERNEL32.dll
 0000:fffd9000       .debug$S                   0000000180000000     kernel32:KERNEL32.dll
 0000:fffd9000       .debug$S                   0000000180000000     kernel32:KERNEL32.dll
 0000:fffd9000       .debug$S                   0000000180000000     kernel32:KERNEL32.dll
 0000:fffd9000       .debug$S                   0000000180000000     kernel32:KERNEL32.dll
 0000:fffd9000       .debug$S                   0000000180000000     kernel32:KERNEL32.dll
 0000:fffd9000       .debug$S                   0000000180000000     kernel32:KERNEL32.dll
 0000:fffd9000       .debug$S                   0000000180000000     kernel32:KERNEL32.dll
 0000:fffd9000       .debug$S                   0000000180000000     kernel32:KERNEL32.dll
 0000:fffd9000       .debug$S                   0000000180000000     kernel32:KERNEL32.dll
 0000:fffd9000       .debug$S                   0000000180000000     kernel32:KERNEL32.dll
 0000:fffd9000       .debug$S                   0000000180000000     kernel32:KERNEL32.dll
 0000:fffd9000       .debug$S                   0000000180000000     kernel32:KERNEL32.dll
 0000:fffd9000       .debug$S                   0000000180000000     kernel32:KERNEL32.dll
 0000:fffd9000       .debug$S                   0000000180000000     kernel32:KERNEL32.dll
 0000:fffd9000       .debug$S                   0000000180000000     kernel32:KERNEL32.dll
 0000:fffd9000       .debug$S                   0000000180000000     kernel32:KERNEL32.dll
 0000:fffd9000       .debug$S                   0000000180000000     kernel32:KERNEL32.dll
 0000:fffd9000       .debug$S                   0000000180000000     kernel32:KERNEL32.dll
 0000:fffd9000       .debug$S                   0000000180000000     kernel32:KERNEL32.dll
 0000:fffd9000       .debug$S                   0000000180000000     kernel32:KERNEL32.dll
 0000:fffd9000       .debug$S                   0000000180000000     kernel32:KERNEL32.dll
 0000:fffd9000       .debug$S                   0000000180000000     kernel32:KERNEL32.dll
 0000:fffd9000       .debug$S                   0000000180000000     kernel32:KERNEL32.dll
 0000:fffd9000       .debug$S                   0000000180000000     kernel32:KERNEL32.dll
 0000:fffd9000       .debug$S                   0000000180000000     kernel32:KERNEL32.dll
 0000:fffd9000       .debug$S                   0000000180000000     kernel32:KERNEL32.dll
 0001:00001218       addRefToVerify             0000000180002218 f   libredefclass030.obj
 0001:0000128c       agentProc                  000000018000228c f   libredefclass030.obj
 0001:000015fc       agentThreadWrapper         00000001800025fc f   libredefclass030.obj
 0001:00001750       check_option               0000000180002750 f   libredefclass030.obj
 0001:00001998       file_basename              0000000180002998 f   libredefclass030.obj
 0001:000025f0       startAgentThreadWrapper    00000001800035f0 f   libredefclass030.obj
 0001:0000291c       syncDebuggeeStatus         000000018000391c f   libredefclass030.obj
 0001:00002ba4       capture_previous_context   0000000180003ba4 f   MSVCRT:gs_report.obj
 0001:00002c18       ?__scrt_initialize_thread_safe_statics@@YAHXZ 0000000180003c18 f   MSVCRT:thread_safe_statics.obj
 0001:00002ce8       ?__scrt_uninitialize_thread_safe_statics@@YAXXZ 0000000180003ce8 f   MSVCRT:thread_safe_statics.obj
 0001:00002d90       $$000000                   0000000180003d90     MSVCRT:amdsecgs.obj
 0001:00002dc0       ?dllmain_crt_dispatch@@YAHQEAUHINSTANCE__@@KQEAX@Z 0000000180003dc0 f   MSVCRT:dll_dllmain.obj
 0001:00002e10       ?dllmain_crt_process_attach@@YAHQEAUHINSTANCE__@@QEAX@Z 0000000180003e10 f   MSVCRT:dll_dllmain.obj
 0001:00002f28       ?dllmain_crt_process_detach@@YAH_N@Z 0000000180003f28 f   MSVCRT:dll_dllmain.obj
 0001:00002fac       ?dllmain_dispatch@@YAHQEAUHINSTANCE__@@KQEAX@Z 0000000180003fac f   MSVCRT:dll_dllmain.obj
 0001:000039c0       $$000000                   00000001800049c0     MSVCRT:guard_dispatch.obj
 0001:000039e0       $$000000                   00000001800049e0     MSVCRT:guard_xfg_dispatch.obj
 0001:000039f6       ?fin$0@?0??dllmain_crt_process_attach@@YAHQEAUHINSTANCE__@@QEAX@Z@4HA 00000001800049f6 f   MSVCRT:dll_dllmain.obj
 0001:00003a0d       ?fin$0@?0??dllmain_crt_process_detach@@YAH_N@Z@4HA 0000000180004a0d f   MSVCRT:dll_dllmain.obj
 0001:00003a26       ?fin$1@?0??dllmain_crt_process_detach@@YAH_N@Z@4HA 0000000180004a26 f   MSVCRT:dll_dllmain.obj
 0001:00003a3a       ?filt$0@?0??dllmain_dispatch@@YAHQEAUHINSTANCE__@@KQEAX@Z@4HA 0000000180004a3a f   MSVCRT:dll_dllmain.obj
 0001:00003a70       __scrt_is_nonwritable_in_current_image$filt$0 0000000180004a70 f   MSVCRT:utility.obj
 0002:00000220       ?__scrt_initialize_tss_var@@3P6AHXZEA 0000000180005220     MSVCRT:thread_safe_statics.obj
 0002:00000340       ?opcLengths@@3QBEB         0000000180005340     libredefclass030.obj
 0002:00002410       GS_ExceptionPointers       0000000180007410     MSVCRT:gs_report.obj
 0002:00002b70       $unwind$fprintf            0000000180007b70     libredefclass030.obj
 0002:00002b7c       $unwind$printf             0000000180007b7c     libredefclass030.obj
 0002:00002b88       $unwind$?NewObject@JNIEnv_@@QEAAPEAV_jobject@@PEAV_jclass@@PEAU_jmethodID@@ZZ 0000000180007b88     libredefclass030.obj
 0002:00002b88       $unwind$nsk_lcomplain      0000000180007b88     libredefclass030.obj
 0002:00002b88       $unwind$nsk_ldisplay       0000000180007b88     libredefclass030.obj
 0002:00002b90       $unwind$nsk_lvdisplay      0000000180007b90     libredefclass030.obj
 0002:00002b90       $unwind$_RTC_Initialize    0000000180007b90     MSVCRT:initsect.obj
 0002:00002b90       $unwind$_RTC_Terminate     0000000180007b90     MSVCRT:initsect.obj
 0002:00002b90       $unwind$?__scrt_initialize_thread_safe_statics@@YAHXZ 0000000180007b90     MSVCRT:thread_safe_statics.obj
 0002:00002b9c       $unwind$nsk_complain       0000000180007b9c     libredefclass030.obj
 0002:00002b9c       $unwind$nsk_printf         0000000180007b9c     libredefclass030.obj
 0002:00002ba4       $unwind$nsk_lvcomplain     0000000180007ba4     libredefclass030.obj
 0002:00002bbc       $unwind$nsk_ltrace         0000000180007bbc     libredefclass030.obj
 0002:00002bbc       $unwind$__report_gsfailure 0000000180007bbc     MSVCRT:gs_report.obj
 0002:00002bc4       $unwind$nsk_lvtrace        0000000180007bc4     libredefclass030.obj
 0002:00002bc4       $unwind$__raise_securityfailure 0000000180007bc4     MSVCRT:gs_report.obj
 0002:00002bc4       $unwind$__scrt_initialize_crt 0000000180007bc4     MSVCRT:utility.obj
 0002:00002bc4       $unwind$__scrt_initialize_onexit_tables 0000000180007bc4     MSVCRT:utility.obj
 0002:00002bc4       $unwind$__scrt_release_startup_lock 0000000180007bc4     MSVCRT:utility.obj
 0002:00002bc4       $unwind$__scrt_uninitialize_crt 0000000180007bc4     MSVCRT:utility.obj
 0002:00002bc4       $unwind$_onexit            0000000180007bc4     MSVCRT:utility.obj
 0002:00002bcc       $unwind$nsk_lverify        0000000180007bcc     libredefclass030.obj
 0002:00002bdc       $unwind$nsk_vprintf        0000000180007bdc     libredefclass030.obj
 0002:00002bec       $unwind$?nsk_jni_lverify@@YAHHPEAUJNIEnv_@@HQEBDH1ZZ 0000000180007bec     libredefclass030.obj
 0002:00002c00       $unwind$?nsk_jni_check_exception@@YAHPEAUJNIEnv_@@QEBDH@Z 0000000180007c00     libredefclass030.obj
 0002:00002c1c       $unwind$nsk_jvmti_parseOptions 0000000180007c1c     libredefclass030.obj
 0002:00002c38       $unwind$nsk_jvmti_createJVMTIEnv 0000000180007c38     libredefclass030.obj
 0002:00002c4c       $unwind$check_option       0000000180007c4c     libredefclass030.obj
 0002:00002c4c       $unwind$nsk_jvmti_waitForSync 0000000180007c4c     libredefclass030.obj
 0002:00002c4c       $unwind$_DllMainCRTStartup 0000000180007c4c     MSVCRT:dll_dllmain.obj
 0002:00002c5c       $unwind$Java_nsk_jvmti_RedefineClasses_redefclass030_isRedefinitionOccurred 0000000180007c5c     libredefclass030.obj
 0002:00002c5c       $unwind$Java_nsk_jvmti_RedefineClasses_redefclass030_notifyNativeAgent 0000000180007c5c     libredefclass030.obj
 0002:00002c5c       $unwind$Java_nsk_jvmti_unit_FollowReferences_FollowRefObjects_resetTags 0000000180007c5c     libredefclass030.obj
 0002:00002c5c       $unwind$addRefToVerify     0000000180007c5c     libredefclass030.obj
 0002:00002c5c       $unwind$nsk_jvmti_resetAgentData 0000000180007c5c     libredefclass030.obj
 0002:00002c5c       $unwind$nsk_jvmti_resumeSync 0000000180007c5c     libredefclass030.obj
 0002:00002c5c       $unwind$__scrt_initialize_default_local_stdio_options 0000000180007c5c     MSVCRT:default_local_stdio_options.obj
 0002:00002c5c       $unwind$?dllmain_crt_dispatch@@YAHQEAUHINSTANCE__@@KQEAX@Z 0000000180007c5c     MSVCRT:dll_dllmain.obj
 0002:00002c5c       $unwind$DllMain            0000000180007c5c     MSVCRT:dll_dllmain_stub.obj
 0002:00002c5c       $unwind$__GSHandlerCheck   0000000180007c5c     MSVCRT:gshandler.obj
 0002:00002c5c       $unwind$?__scrt_uninitialize_thread_safe_statics@@YAXXZ 0000000180007c5c     MSVCRT:thread_safe_statics.obj
 0002:00002c5c       $unwind$__scrt_acquire_startup_lock 0000000180007c5c     MSVCRT:utility.obj
 0002:00002c5c       $unwind$__scrt_dllmain_after_initialize_c 0000000180007c5c     MSVCRT:utility.obj
 0002:00002c5c       $unwind$__scrt_dllmain_before_initialize_c 0000000180007c5c     MSVCRT:utility.obj
 0002:00002c5c       $unwind$__scrt_dllmain_crt_thread_attach 0000000180007c5c     MSVCRT:utility.obj
 0002:00002c5c       $unwind$__scrt_dllmain_crt_thread_detach 0000000180007c5c     MSVCRT:utility.obj
 0002:00002c5c       $unwind$__scrt_dllmain_uninitialize_c 0000000180007c5c     MSVCRT:utility.obj
 0002:00002c5c       $unwind$__scrt_dllmain_uninitialize_critical 0000000180007c5c     MSVCRT:utility.obj
 0002:00002c5c       $unwind$atexit             0000000180007c5c     MSVCRT:utility.obj
 0002:00002c64       $unwind$nsk_jvmti_enableEvents 0000000180007c64     libredefclass030.obj
 0002:00002c7c       $unwind$nsk_jvmti_lverify  0000000180007c7c     libredefclass030.obj
 0002:00002c90       $unwind$exitOnError        0000000180007c90     libredefclass030.obj
 0002:00002ca0       $unwind$Java_nsk_share_jvmti_ArgumentHandler_getAgentOptionsString 0000000180007ca0     libredefclass030.obj
 0002:00002cb4       $unwind$Java_nsk_jvmti_unit_FollowReferences_FollowRefObjects_getTag 0000000180007cb4     libredefclass030.obj
 0002:00002cb4       $unwind$Java_nsk_share_jvmti_DebugeeClass_checkStatus 0000000180007cb4     libredefclass030.obj
 0002:00002cb4       $unwind$agentThreadWrapper 0000000180007cb4     libredefclass030.obj
 0002:00002cc4       $unwind$startAgentThreadWrapper 0000000180007cc4     libredefclass030.obj
 0002:00002ce0       $unwind$syncDebuggeeStatus 0000000180007ce0     libredefclass030.obj
 0002:00002ce0       $unwind$__scrt_dllmain_exception_filter 0000000180007ce0     MSVCRT:utility.obj
 0002:00002cf4       $unwind$Java_nsk_share_jvmti_DebugeeClass_resetAgentData 0000000180007cf4     libredefclass030.obj
 0002:00002cfc       $unwind$MA_checkStatus     0000000180007cfc     libredefclass030.obj
 0002:00002d10       $unwind$Java_nsk_jvmti_unit_FollowReferences_FollowRefObjects_setTag 0000000180007d10     libredefclass030.obj
 0002:00002d28       $unwind$Java_nsk_jvmti_unit_FollowReferences_FollowRefObjects_addRefToVerify 0000000180007d28     libredefclass030.obj
 0002:00002d44       $unwind$Agent_Initialize   0000000180007d44     libredefclass030.obj
 0002:00002d68       $unwind$Java_nsk_jvmti_RedefineClasses_redefclass030_storeClassBytes 0000000180007d68     libredefclass030.obj
 0002:00002d74       $unwind$CompiledMethodLoad 0000000180007d74     libredefclass030.obj
 0002:00002d8c       $unwind$CompiledMethodUnload 0000000180007d8c     libredefclass030.obj
 0002:00002d9c       $unwind$agentProc          0000000180007d9c     libredefclass030.obj
 0002:00002db4       $unwind$capture_previous_context 0000000180007db4     MSVCRT:gs_report.obj
 0002:00002dc0       $unwind$__GSHandlerCheckCommon 0000000180007dc0     MSVCRT:gshandler.obj
 0002:00002dc8       $xdatasym                  0000000180007dc8     MSVCRT:amdsecgs.obj
 0002:00002dcc       $unwind$?dllmain_crt_process_attach@@YAHQEAUHINSTANCE__@@QEAX@Z 0000000180007dcc     MSVCRT:dll_dllmain.obj
 0002:00002e08       $unwind$?fin$0@?0??dllmain_crt_process_attach@@YAHQEAUHINSTANCE__@@QEAX@Z@4HA 0000000180007e08     MSVCRT:dll_dllmain.obj
 0002:00002e08       $unwind$?fin$0@?0??dllmain_crt_process_detach@@YAH_N@Z@4HA 0000000180007e08     MSVCRT:dll_dllmain.obj
 0002:00002e08       $unwind$?fin$1@?0??dllmain_crt_process_detach@@YAH_N@Z@4HA 0000000180007e08     MSVCRT:dll_dllmain.obj
 0002:00002e10       $unwind$?dllmain_crt_process_detach@@YAH_N@Z 0000000180007e10     MSVCRT:dll_dllmain.obj
 0002:00002e64       $unwind$?dllmain_dispatch@@YAHQEAUHINSTANCE__@@KQEAX@Z 0000000180007e64     MSVCRT:dll_dllmain.obj
 0002:00002e8c       $unwind$?filt$0@?0??dllmain_dispatch@@YAHQEAUHINSTANCE__@@KQEAX@Z@4HA 0000000180007e8c     MSVCRT:dll_dllmain.obj
 0002:00002e94       $unwind$__scrt_is_nonwritable_in_current_image 0000000180007e94     MSVCRT:utility.obj
 0002:00002eb4       $unwind$__scrt_is_nonwritable_in_current_image$filt$0 0000000180007eb4     MSVCRT:utility.obj
 0002:00002ebc       $unwind$__scrt_fastfail    0000000180007ebc     MSVCRT:utility_desktop.obj
 0002:00002ecc       $unwind$__security_init_cookie 0000000180007ecc     MSVCRT:gs_support.obj
 0002:00002ed8       $unwind$__isa_available_init 0000000180007ed8     MSVCRT:cpu_disp.obj
 0002:00002ee8       $xdatasym                  0000000180007ee8     MSVCRT:guard_dispatch.obj
 0002:00002ef0       $xdatasym                  0000000180007ef0     MSVCRT:guard_xfg_dispatch.obj
 0002:00002f00       .edata                     0000000180007f00     redefclass030.exp
 0002:00002f28       rgpv                       0000000180007f28     redefclass030.exp
 0002:00002f70       rgszName                   0000000180007f70     redefclass030.exp
 0002:00002fb8       rgwOrd                     0000000180007fb8     redefclass030.exp
 0002:00002fdc       szName                     0000000180007fdc     redefclass030.exp
 0002:00002fee       $N00001                    0000000180007fee     redefclass030.exp
 0002:00002ffd       $N00002                    0000000180007ffd     redefclass030.exp
 0002:0000300a       $N00003                    000000018000800a     redefclass030.exp
 0002:0000301f       $N00004                    000000018000801f     redefclass030.exp
 0002:00003063       $N00005                    0000000180008063     redefclass030.exp
 0002:000030a2       $N00006                    00000001800080a2     redefclass030.exp
 0002:000030df       $N00007                    00000001800080df     redefclass030.exp
 0002:00003124       $N00008                    0000000180008124     redefclass030.exp
 0002:00003161       $N00009                    0000000180008161     redefclass030.exp
 0002:000031a9       $N00010                    00000001800081a9     redefclass030.exp
 0002:000031e9       $N00011                    00000001800081e9     redefclass030.exp
 0002:00003226       $N00012                    0000000180008226     redefclass030.exp
 0002:00003261       $N00013                    0000000180008261     redefclass030.exp
 0002:0000328f       $N00014                    000000018000828f     redefclass030.exp
 0002:000032c0       $N00015                    00000001800082c0     redefclass030.exp
 0002:000032ef       $N00016                    00000001800082ef     redefclass030.exp
 0002:0000331e       $N00017                    000000018000831e     redefclass030.exp
 0002:00003353       $N00018                    0000000180008353     redefclass030.exp
 0002:000037ca       .idata$6                   00000001800087ca     kernel32:KERNEL32.dll
 0002:0000382e       .idata$6                   000000018000882e     vcruntime:VCRUNTIME140.dll
 0002:000039c0       .idata$6                   00000001800089c0     ucrt:api-ms-win-crt-heap-l1-1-0.dll
 0002:000039e0       .idata$6                   00000001800089e0     ucrt:api-ms-win-crt-runtime-l1-1-0.dll
 0002:00003a02       .idata$6                   0000000180008a02     ucrt:api-ms-win-crt-convert-l1-1-0.dll
 0002:00003a24       .idata$6                   0000000180008a24     ucrt:api-ms-win-crt-stdio-l1-1-0.dll
 0002:00003a44       .idata$6                   0000000180008a44     ucrt:api-ms-win-crt-string-l1-1-0.dll
 0003:00000000       ?codeAttributeName@@3PEBDEB 0000000180009000     libredefclass030.obj
 0003:00000008       ?lineNumberAttributeName@@3PEBDEB 0000000180009008     libredefclass030.obj
 0003:00000010       ?localVarAttributeName@@3PEBDEB 0000000180009010     libredefclass030.obj
 0003:00000018       ?localVarTypeAttributeName@@3PEBDEB 0000000180009018     libredefclass030.obj
 0003:00000020       ?stackMapAttributeName@@3PEBDEB 0000000180009020     libredefclass030.obj
 0003:00000028       ?callBytes@@3PAEA          0000000180009028     libredefclass030.obj
 0003:0000002c       ?allocBytes@@3PAEA         000000018000902c     libredefclass030.obj
 0003:00000030       expHSMethod                0000000180009030     libredefclass030.obj
 0003:00000038       expHSSignature             0000000180009038     libredefclass030.obj
 0003:00000040       eventsList                 0000000180009040     libredefclass030.obj
 0003:0001aae4       redefineAttempted          0000000180023ae4     libredefclass030.obj
 0003:0001aae8       nsk_context                0000000180023ae8     libredefclass030.obj
 0003:0001aaf4       redefineSucceed            0000000180023af4     libredefclass030.obj
 0003:0001aaf8       agentFailed                0000000180023af8     libredefclass030.obj
 0003:0001aafc       currentAgentStatus         0000000180023afc     libredefclass030.obj
 0003:0001ab00       context                    0000000180023b00     libredefclass030.obj
 0003:0001abb8       agentThread                0000000180023bb8     libredefclass030.obj
 0003:0001abc0       agentThreadProc            0000000180023bc0     libredefclass030.obj
 0003:0001abc8       agentThreadArg             0000000180023bc8     libredefclass030.obj
 0003:0001abd0       agent_data                 0000000180023bd0     libredefclass030.obj
 0003:0001abe0       jvmti_env                  0000000180023be0     libredefclass030.obj
 0003:0001abe8       jvm                        0000000180023be8     libredefclass030.obj
 0003:0001abf0       jni_env                    0000000180023bf0     libredefclass030.obj
 0003:0001abf8       checkStatus_func           0000000180023bf8     libredefclass030.obj
 0003:0001ac00       ?codeAttributeIndex@@3GA   0000000180023c00     libredefclass030.obj
 0003:0001ac04       ?lineNumberAttributeIndex@@3GA 0000000180023c04     libredefclass030.obj
 0003:0001ac08       ?localVarAttributeIndex@@3GA 0000000180023c08     libredefclass030.obj
 0003:0001ac0c       ?localVarTypeAttributeIndex@@3GA 0000000180023c0c     libredefclass030.obj
 0003:0001ac10       ?stackMapAttributeIndex@@3GA 0000000180023c10     libredefclass030.obj
 0003:0001ac14       ?stackFrameOffset@@3GA     0000000180023c14     libredefclass030.obj
 0003:0001ac18       ?mode@@3HA                 0000000180023c18     libredefclass030.obj
 0003:0001ac1c       ?constantPoolSize@@3GA     0000000180023c1c     libredefclass030.obj
 0003:0001ac20       ?orig@@3PEBEEB             0000000180023c20     libredefclass030.obj
 0003:0001ac28       ?gen@@3PEAEEA              0000000180023c28     libredefclass030.obj
 0003:0001ac30       ?inputPos@@3PEAEEA         0000000180023c30     libredefclass030.obj
 0003:0001ac38       ?endPos@@3PEBEEB           0000000180023c38     libredefclass030.obj
 0003:0001ac40       ?genPos@@3PEAEEA           0000000180023c40     libredefclass030.obj
 0003:0001ac48       ?markPos@@3PEAEEA          0000000180023c48     libredefclass030.obj
 0003:0001ac50       ?constantPool@@3PEAPEADEA  0000000180023c50     libredefclass030.obj
 0003:0001ac58       ?constantPoolCount@@3GA    0000000180023c58     libredefclass030.obj
 0003:0001ac5c       ?zeroBytes@@3PAEA          0000000180023c5c     libredefclass030.obj
 0003:0001ac60       ?codeLength@@3IA           0000000180023c60     libredefclass030.obj
 0003:0001ac64       fire                       0000000180023c64     libredefclass030.obj
 0003:0001ac68       ?map@@3PEAIEA              0000000180023c68     libredefclass030.obj
 0003:0001ac70       ?widening@@3PEACEA         0000000180023c70     libredefclass030.obj
 0003:0001ac78       jvmti                      0000000180023c78     libredefclass030.obj
 0003:0001ac80       timeout                    0000000180023c80     libredefclass030.obj
 0003:0001ac88       hsMethodID                 0000000180023c88     libredefclass030.obj
 0003:0001ac90       enteredHotMethod           0000000180023c90     libredefclass030.obj
 0003:0001ac94       bytesCount                 0000000180023c94     libredefclass030.obj
 0003:0001ac98       clsBytes                   0000000180023c98     libredefclass030.obj
 0003:0001acb0       GS_ExceptionRecord         0000000180023cb0     MSVCRT:gs_report.obj
 0003:0001ad50       GS_ContextRecord           0000000180023d50     MSVCRT:gs_report.obj
 0003:0001b220       ?g_tss_cv@@3U_RTL_CONDITION_VARIABLE@@A 0000000180024220     MSVCRT:thread_safe_statics.obj
 0003:0001b228       ?g_tss_event@@3PEAXEA      0000000180024228     MSVCRT:thread_safe_statics.obj
 0003:0001b230       ?g_tss_mutex@@3U_RTL_CRITICAL_SECTION@@A 0000000180024230     MSVCRT:thread_safe_statics.obj
 0003:0001b258       ?g_sleep_condition_variable_cs@@3P6AHPEAU_RTL_CONDITION_VARIABLE@@PEAU_RTL_CRITICAL_SECTION@@K@ZEA 0000000180024258     MSVCRT:thread_safe_statics.obj
 0003:0001b260       ?g_wake_all_condition_variable@@3P6AXPEAU_RTL_CONDITION_VARIABLE@@@ZEA 0000000180024260     MSVCRT:thread_safe_statics.obj
 0003:0001b26c       ?__proc_attached@@3HA      000000018002426c     MSVCRT:dll_dllmain.obj
 0003:0001b280       ?is_initialized_as_dll@@3_NA 0000000180024280     MSVCRT:utility.obj
 0003:0001b281       ?module_local_atexit_table_initialized@@3_NA 0000000180024281     MSVCRT:utility.obj
 0003:0001b288       ?module_local_atexit_table@@3U_onexit_table_t@@A 0000000180024288     MSVCRT:utility.obj
 0003:0001b2a0       ?module_local_at_quick_exit_table@@3U_onexit_table_t@@A 00000001800242a0     MSVCRT:utility.obj
